:030000000219FDE5
:03000B000200AA46
:03002B0002015C73
:03005B000202EBB3
:030073000202D8AE
:1000800002030406080C10182030406080040608A3
:100090000C10182030406080A0C00003070F1F0D17
:1000A0000D0403060D0503030202C2AFC0D0C0E079
:1000B000206214E5256009E473E525F4F58AD2622F
:1000C000D0E0D0D0D2AF3285268AC262E526F46075
:1000D0002F30682520720DD0E0D0D0D292D291D2AC
:1000E00090D2AF32D292D291D290206F0C2066097A
:1000F000740AD5E0FDE57B4290D0E0D0D0D2AF329B
:10010000758A00C28DD26201F901B9306805206696
:1001100002C29201B9306805206602C29101B9306D
:100120006805206602C29001B9C29330680A206651
:10013000077408D5E0FDC29201B9C29430680A2064
:1001400066077408D5E0FDC29101B9C29530680A0E
:100150002066077408D5E0FDC29001B9C2AFC2ADF8
:1001600053E6EFC0D0C0E0D2D3D2AFC2CEE52A6012
:1001700007207449152A21BD7800790020742EE5E6
:1001800080307E01F430E40278FF53DACF207E0322
:1001900043DA20307E0343DA10C2D8C271E58030E2
:1001A0007E01F430E40279FFC3E89970CB3061033B
:1001B000752A40207403752A40885CD27020740D23
:1001C000E52B6004152B21CD43DA01C2D820700243
:1001D00021E0A85C206102C27020740221DE882226
:1001E0007882B60403852224C3E52594404002D2D8
:1001F0006420CF0AD0E0D0D043E610D2AD32C2CFD7
:10020000053A7802E52A6005307402152AC3E55CD8
:1002100094014005755F00412A756000756900E52D
:100220005F2401F55F5003755FFF7982B7020D30DF
:100230006E1DC3E52294324016854C227982B703A5
:100240000E306E0BC3E52294324004798E8722C3B0
:10025000E5239522600840041523415E0523D8CA92
:100260000569E56970021569D56A63756A017805E3
:10027000C3E569956B4057C3E569956C50087801F3
:10028000756A03020292C3E569956D5005780175A0
:100290006A01C3E5629524401E7982B7040241C316
:1002A000206E14852462E569046003856B69756AB4
:1002B0000175233C0202CEE5622850057562FF41BC
:1002C000C3F562E5620470067560FF7569FFD0E0F2
:1002D000D0D043E610D2AD32C2AF53E67F7592FA6A
:1002E0007593FFC260759104D2AF32C2AF53E6EF8F
:1002F000C2ADC0D0C0E0C0F0D2D3D2AFA8FBA9FC41
:10030000C2D8307102615253DACF207E0343DA1033
:10031000307E0343DA20D271E580307E01F420E4A0
:1003200002612988278928A13753DACF207E034329
:10033000DA20307E0343DA10C2D8C271307402A1D1
:10034000237800E580307E01F430E402A123885C4C
:10035000A10B53DACF207E0343DA20307E0343DA49
:1003600010C271206102812B53DACF207E0343DA61
:1003700010307E0343DA20C2D8D27188578958C31F
:10038000E89555F8E99556F97B007E087A00C3E8B0
:10039000948CE994005005755B00811D882178A23A
:1003A000E6A8216055C3E894C8E994005008E4D257
:1003B000E4FB7A0A61F8C3E89468E994015008E420
:1003C000D2E3FB7A0F61F8C3E894D0E994025008B5
:1003D000E4D2E2FB7A1E61F8C3E894A0E9940550E8
:1003E00008E4D2E1FB7A3C61F8C3E89498E9940808
:1003F0005008E4D2E0FB7A787E00C3E89559FCE926
:10040000955AFD30E70AECF42401FCEDF43400FDCC
:10041000755B00C3EC9AED9E5003755B01885989AA
:100420005A8557558558567802A10BC3E89527F889
:10043000E99528F9307C0281EF307B0281EF307A38
:100440000281E8207502814EE9FDE8FC816DE9C377
:1004500013F9E813F830790281E8E9C313F9E813D6
:10046000F830780281E8E9C313FDE813FC20612C21
:0F047000C3EC941CED940240028184ED701EC316
:10047F00EC94C850180529E52970021529C3E52900
:10048F00940A5002A123755C00D270A123E5296064
:10049F000215297400207F037896E624FAFEE434CF
:1004AF0000FFC3EC9EFCED9FFD50067800790081A4
:1004BF00EFC3EC94FFED9400400678FF790081EFD5
:1004CF00EC8572F0A4C5F0A2F733F879004003026F
:1004DF00050B78FF790002050BE9C313F9E813F850
:1004EF00307C0EE9600278FFC3E81338F8E434007B
:1004FF00F9C3E894FFE99400400278FF885CD2705A
:10050F00206102A123741FF4552F4BF52FC274EBFA
:10051F007002D274752A40307403752A0A30610252
:10052F00A13720740353DAFE207403752B20D0F00B
:10053F00D0E0D0D0D2AD43E6103279010205677911
:10054F0003020567790A020567791E020567796458
:10055F0002056779C80205677817E4D5E0FDD8FA78
:10056F00D9F6227A147B7802058E7A107B8C0205DD
:10057F008E7A0D7BB402058E7A0B7BC802058E79BD
:10058F0002E4C294D5E0FDC291D5E0FDD291D5E051
:10059F00FDD294D5E0FDE920E002C29230E002C224
:1005AF0090E573D5E0FDE920E002D29230E002D26F
:1005BF00907496D5E0FDD9C9EAF8D5E0FDD8FBDBFC
:1005CF00BEC29422C37C007D0075F00005F0EA33B3
:1005DF00FAEB33FB50F6EB13FBEA13FAC3E9FFE830
:1005EF00FEE89AF8E99BF95004EFF9EEF8B3EC3313
:1005FF00FCED33FDD5F0DFEDF9ECF822E889F08A58
:10060F0020D2D4F8A9F07B0030F70B7BFFF4240144
:10061F00F8E9F43400F9E88520F0A4ADF0F8E985A5
:10062F0020F0A4AFF0FEED2EF974003FFA7C04C366
:10063F00EA13FAE913F9E813F8DCF48BF030F70A50
:10064F00E8F42401F8E9F43400F9E889F0C2D4F8A9
:10065F00A9F0227882B60403020701C3E55C94195E
:10066F00401EE52D54067018206E3678057994E7F4
:10067F00146007780A1460027812C3E54198401F8E
:10068F00306E098564627569FF756A01852224E4FD
:10069F00F544F545F546F547F548C26E020701D218
:1006AF006E7994E7147013E523F43333F913F8E9F3
:1006BF00540104F9E854FE0206F5E714147014E52A
:1006CF0023F4333333F913F8E9540304F9E854FCF2
:1006DF000206FDE523F433333333F913F8E95407F6
:1006EF000404F9E854F8C39440F8E99400F98844F5
:1006FF00894522C3E54113F9E54013F8C3E5449852
:10070F00F8E54599F9500CC3E89480E994FF401639
:10071F00020739C3E8947FE9940050030207397840
:10072F007F7900020739788079FF8849894A22E565
:10073F00492546F8E54A3547F9854A20E43007014F
:10074F00F43548FA30E709C3EA94F0401502077709
:10075F00C3EA940F500302077778FF79FF7A0F02ED
:10076F000777780079007AF0C3E5249561500AC3C2
:10077F0074019524500B020795E54A20E70E0207F6
:10078F0095E54A30E706884689478A482278A5E6E4
:10079F00FAC3E54933F8E54A33F9D10BE930E70BF2
:1007AF00C3E89480E994FF4013E1CFC3E8947FE955
:1007BF0094005002E1CF787F7900E1CF788079FF04
:1007CF00E820E715C3E52398F84009C3E8940140F2
:1007DF00030207F678010207F6E8F424012523F84F
:1007EF0040030207F678FF884B2278A6E6FAA8475F
:1007FF00A94812060BE930E70CC3E89401E994FF0E
:10080F00401602082BC3E894FFE994005003020836
:10081F002B78FF790002082B780179FFE920E71583
:10082F00C3E54B98F84009C3E8940140030208520E
:10083F007801020852E8F42401254BF8400302081E
:10084F005278FF88242278FFC26420693D206A1203
:10085F00D264C3E541940A4009C3E5259440500290
:0D086F00C26479A1E76023E541601F74FFBA
:10087C008541F0848539F0306A0375F005A4F8C51C
:10088C00F0600278FFC3E895645002A86488632284
:10089C00C3E5409440E5419401E56350031401AD78
:1008AC00046002F563227883E6F520120F2A75E8BE
:1008BC009012054975E890E5E820ECFBA8BDA9BEAF
:1008CC00120FD0756EAF756F00C3740013FD74AF4B
:1008DC00606613FC74AF2CFC74003DFDECFAEDFB70
:1008EC00C3E89AE99B4014E56E24AFF56EE56F34CE
:1008FC0000F56FEA2CFAEB3DFB80E5AE6EAF6FC3F3
:10090C00E56F13F9E56E13F8C3E913F9E813F87AF8
:10091C0003C3E913F9E813F8DAF7AA201A7009757A
:10092C006E00756F000209441AEA6008EE28FEEFAB
:10093C0039FFDAF88E6E8F6F2275E890227883E695
:10094C00FFE5E820ECF7A8BDA9BE0570C3E57094DF
:10095C00084052757000E9FA79A0E76044EA700724
:10096C00E571601B02097FC3E895716010E5715059
:10097C0006600C1402098B0460F902098BE571F511
:10098C0071C39458401B7561C0C3940440137561C6
:10099C0080C39404400B756140C39404400375619B
:1009AC000075BB0322EFC39401601F74AF601BC3BF
:1009BC00E894FFE994035012C3E8956EE9956F50E3
:1009CC0009E561600C15610209DDE561F460020561
:1009DC0061A861C3E524985002A824C3E89562403D
:1009EC000AA862E562F4600385626188258826E5C1
:1009FC0070B4070375BB1022743279A787F0A4C5B5
:100A0C00F0A2F733F8C3E895614002A86188228808
:100A1C0024882588268864227540007541F022C2FE
:100A2C00AF75C820A8CCA9CDAA3A30CF010A75C899
:100A3C0024D2AFAB3BAC3C883B893CC3E89BF8E988
:100A4C009C206908F930670261374194AD3D8A3DBD
:100A5C00F9EA9DFA600478FF79FFAE3EAF3F8B3E1A
:100A6C008C3FA83BA93CC3E89EF8E99FF9C3E5413C
:100A7C0013FBE54013FAE82AF540E93BF541500633
:100A8C007540FF7541FF41DEAA40AB41AC40AD4122
:100A9C007E047F02C3EB940440021E1FC3EB940838
:100AAC0040021E1FC3ED13FDEC13FCDEF7C3EA9CE2
:100ABC00FAEB9DFBEF6009C3E913F9E813F8DFF7D4
:100ACC00EA28FAEB39FB8A408B4150067BFF8B40BE
:100ADC008B41C3EB94025002D2673069047F0361EF
:100AEC00097892E6FFC3E537948240110FC3E537CE
:100AFC0094A040010FC3EF940640027F057E02E5EF
:100B0C0041C4540FF9E541C454F0F8E540C4540F06
:100B1C0028F8C3E89EFAE99400FB4009C3EA940262
:100B2C00EB940050047A02E4FB6183AA40AB41EBE6
:100B3C00C4FEEAC4540F4EFCC3EA9CFAEB9400FBCF
:100B4C00C3E813C313F8EA28FAEB3400FB8A408B92
:100B5C0041C3EB94024002C2677802EBC4FE7B00F7
:100B6C00EAC4540F4EFAC3EA98FA4005C3940250F3
:100B7C00027A027892E6FF30600261838551928599
:100B8C005293D26043E680C3E49AF8E49BF9306751
:100B9C0002810FE8FAE9FBD3E913FDE813FC885155
:100BAC008952C3EF94036038EF20E00DE82CF8E98C
:100BBC003DF9ECFAEDFB020BD8E828F8E939F9C35A
:100BCC00E82402F8E93400F97AFE7BFFC3EF9403C2
:100BDC00400E8A538B54884D894E8C4F8D508143D7
:100BEC00885389548A4D8B4E8C4F8D5030691275B9
:100BFC0053F07554FF754FF07550FF7551F07552E9
:100C0C00FF8143E8FAD3E813FC8851C3EF940360E7
:100C1C0020EF20E007E82CF8ECFA812FE8282402DA
:100C2C00F87AFEC3EF940340088A53884D8C4F81A9
:100C3C004388538A4D8C4FE568C3335002646BF57F
:100C4C0068306002814D753402D26043E680E52D38
:100C5C0054066034A840A941C3E913F9E813F8C35A
:0F0C6C00E913F9E813F8306904E92440F9C2AF3D
:100C7B0053E67F759100C3E498F594E499F5957567
:100C8B009104D26043E680D2AF22D26575430075E2
:100C9B002000306C03752040020CB4D26575430004
:100CAB00752040306C037520007801790120672096
:100CBB00E52D54066002C2657914E541C31370013A
:100CCB0004F8C3941440027814306904781B791B20
:100CDB00206010E543600C306903D53404D26DA15C
:100CEB005791550543E59BF45440B52002A1413083
:100CFB00690908C3E89940011881DB20650A08C31C
:100D0B00E899400281B481DBC265C2AF53E67F75BF
:100D1B0091003067127594007595FE759104D26041
:100D2B0043E680D2AF81B4AE40AF41C3E49EF594AD
:100D3B00E49FF595A126C3E5339401500281B430AD
:100D4B00650281B4D802A15581DBC26DC2AF53E6F7
:100D5B007F759100855394855495759104854D92BB
:100D6B00854E93D26043E680D2AFE52D54066008E2
:100D7B00206A020533020D93306D0D206C0A20653D
:100D8B00071581158102160E227800306405306537
:100D9B00027801E53775F007A4F9E5F028F5F0E9DD
:100DAB00A2F013A2F113A2F213F537C394785003F8
:100DBB00753778C3E53795384008D266D292D29111
:100DCB00D290306002A1CD854F92855093D2604373
:100DDB00E68022207D16C2AF754202C294D29330B8
:100DEB006202C290D2AF759F10020FCDC2AF754297
:100DFB0002C294D295306202C292D2AF759F10029A
:100E0B000FCD307243207D20C2AF75420390013A63
:100E1B00757B10D290C295306204C291C12BD294D3
:100E2B00D2AF759F20020FCDC2AF75420390013A2E
:100E3B00757B10D292C293306204C291C14BD29493
:100E4B00D2AF759F00020FCD207D17C2AF75420345
:100E5B00900115D290306202C291D2AF759F2002E1
:100E6B000FCDC2AF754203900115D292306202C210
:100E7B0091D2AF759F00020FCD207D16C2AF754288
:100E8B0004C293D295306202C291D2AF759F000219
:100E9B000FCDC2AF754204C295D293306202C2919C
:100EAB00D2AF759F20020FCD307243207D20C2AF91
:100EBB00754205900129757B08D291C2943062046A
:100ECB00C292C1D1D293D2AF759F10020FCDC2AFD8
:100EDB0075420590014B757B20D291C29430620410
:100EEB00C290C1F1D295D2AF759F10020FCD207D6C
:100EFB0017C2AF75420590010BD291306202C292BC
:100F0B00D2AF759F10020FCDC2AF75420590011F76
:100F1B00D2913062EBC290D2AF759F10020FCD20F1
:100F2B007D16C2AF754206C295D294306202C29250
:100F3B00D2AF759F20020FCDC2AF754206C293D2BE
:100F4B0094306202C290D2AF759F00020FCD307207
:100F5B0043207D20C2AF75420190014B757B20D29F
:100F6B0092C293306204C290E177D295D2AF759F53
:100F7B0000020FCDC2AF754201900129757B08D2DB
:100F8B0090C295306204C292E197D293D2AF759F13
:100F9B0020020FCD207D17C2AF75420190011FD2E9
:100FAB0092306202C290D2AF759F00020FCDC2AFDA
:100FBB0075420190010BD290306202C292D2AF7592
:100FCB009F20C26622900109757B00D292D291D2EA
:100FDB0090C293C294C295C262227880760708763B
:100FEB00070876010876040876FF0876FF0876096D
:100FFB00087602087601087601788C76010876006F
:10100B000876B40876FF0876FF0876FF08760308A3
:10101B0076FF0876010876FF0876250876D00876E5
:10102B00780876C80876040876FF087601087600FB
:10103B0008767A08760A08760108760108760008A1
:10104B0076FF087600227887E6FFC272BF0302D2D2
:10105B00727888C27DE630E102D27DC27E7889E665
:0E106B0030E102D27EC3EF94026008758E0160
:10107900D273021083758E00C273227880E61490B1
:1010890000809378A5F67881E6149000809378A67D
:10109900F67886E61490008D9378A7F6789FE6F89F
:1010A900700108C3E8941140027811E82828F56B0B
:1010B900256B256B28F56C256B2828F56D7886E658
:1010C900F539C394025003753902789CE67538FFE7
:1010D900B402037538A0B4030375388278A3E61403
:1010E90090009A93F566120FD022227896E6FA7844
:1010F90097E6FB7888E6B40305C3EB940EFB307FD3
:10110900047A007BFFC3EB9AFCC3948250027C8271
:101119007572000572EC8572F0A4C3E5F0947D4008
:10112900F222D27F11F41205587A007B007C10124A
:10113900054EE55C2AFA74003BFBDCF37C04C3EB47
:1011490013FBEA13FADCF7FEC27F11F422E5EF2064
:10115900E6037520000520903FFFE5201460069006
:101169001DFF1460009304600375EF1253D9BF7516
:1011790081C043FF8012054975EF0243B203E5B30D
:10118900240220E70DF521E5E320E0068521B3439C
:10119900E301120FD07580FF75A40075F1D475D4E1
:1011A900EF75908775A54075F2FF75D5BF75A601D6
:1011B90075E24275DB4675EA02120FD0E4F8F6D8FB
:1011C900FD756801120FE5121665789886737530FA
:1011D90001C2AF1205621205721205581205791281
:1011E9000558120580120558121788120562120552
:1011F9006212055DC2AF78FA79FA308407D9FBD853
:10120900F7021C001151118411F311F478988673B7
:10121900120FD075881075890275C82475910475E7
:10122900D84075A82275B80275E690759B80759DA2
:101239000075D10E75BC5875BB0375BA1175E88078
:10124900120549D2AF1208B275360053DACF207EA3
:101259000343DA20307E0343DA1043DA01C2D8C2ED
:1012690071120562D2617B037A0CE55B70077A0C17
:10127900DB030211FD1205582070030211FDC27033
:10128900E55CC3940240E1E52F541F855E5DF55E80
:10129900B55DD5DAD5C26153DACF207E0343DA20B2
:1012A900307E0343DA10C2D8C27178A2E67008D240
:1012B90074E52F54E0F52FC27575290012055D30CC
:1012C9007409C3E529940A4002D27512054E7802C1
:1012D9003074027800C3E55C9840F0C2AF12057221
:1012E900120572120572D2AF120562754C00120511
:1012F9004E788CE6C3940150030213CDE530C394B4
:101309000150030213CD207435C3E55C94FF5003EB
:101319000213CDC2AF120587D2AF12055DC3E55CDA
:10132900940150EFC2AF120572120553120572D221
:10133900AF12055DC3E55C94FF40E902180D7F0516
:10134900D27F11F412055DC2AFC27F11F4AE5CC346
:10135900E55C947FD2AF4076120549C2AF1205878A
:10136900D2AFDFDC312BC3EE94057897F612056214
:101379001216A71217907F0AD27F11F412055DC2C7
:10138900AFC27F11F4AE5CC3E55C947FD2AF50E687
:10139900120549C2AF120572120553120572D2AF76
:1013A900DFD6312BEE24037896F61205621216A7C2
:1013B9001217BF12055D11F4C3E55C94FF50026179
:1013C9000F02180DC3E55C954C4003855C4C120572
:1013D9005D78017988E7B403027805C3E55C984034
:1013E9000241F7C2AF120587120587120587D2AFEE
:1013F900120562753000E4F531F5320531E531F455
:10140900703F0532789AE6781914601278321460C0
:101419000D787D14600878FA146003753200C3E50D
:101429003298401D120FD0120549153275310078D6
:10143900998673C2AF120587D2AF78988673120561
:101449005D120553E52A700530740221FD780120EB
:1014590074027806C3E55C9840A112055DE52A701F
:0E146900030211FDC2AF120FD0E4F522F523ED
:10147700F524F525F526F567D2AF7885E6C333F56C
:1014870065E4F544F545F546F547F548F570F52C5F
:10149700F52DF53775700875BB101205491209450A
:1014A700E5E820ECFBA8BDA9BEE97001F888711238
:1014B700094975700875BB101151C2AF7561FF12EC
:1014C7000A04852261852262852263D2AF752201D3
:1014D700752401752501752601856069756A01788E
:1014E70088E6B40307C27D307602D27DD268D2691E
:1014F700753300120F2A120F59120A24120A2B12DF
:101507000A24120A2B120A24120CA6120662120DC2
:1015170094120DDE120A2B120C95306E031207027D
:1015270020670312085530670312089C120D9412A6
:101537000E0D120A2B120CA6306E0312073E120D67
:1015470094120E84120A2B120C95306E0312079C0C
:10155700120D94120EB3120A2B120CA6306E031240
:1015670007F9120D94120F2A120A2B120945120CB1
:1015770095120D94120F59120949120A2B30692C32
:10158700856461856462856069756A0179187A0C7A
:10159700C3E533994009C269D26A8A350215B3C3D4
:1015A700E55C9401400302150F021616306A1D20F0
:1015B7006C1AE535147006C26AD26BA10FF535C3F4
:1015C700E55C9401400302150F021616753600C339
:1015D700E55F94014009856462856069756A0178F1
:1015E700FA79A4E760027803C3E55F985021307465
:1015F70004E52A601A78F0306C058564617820C3A9
:10160700E541985002A10F0536E55C6002C11975E6
:101617003600C2AF120FD07887E6FE7602115178F6
:1016270087EEF6E4F522F523F524F525F526F5658D
:10163700752C00752D00D2AF12055D120FD078A45E
:10164700E66006C292C291C290307406E52A700223
:1016570021FD788DE6C39401400241D461FF901AC1
:101667000D78201216E9E520B4A50CA31216E9E5BA
:1016770020B45A03021687120FE51216A70216A600
:10168700901A0378807B0A1216E9A308DBF9901AEF
:101697000F788C7B191216E9A308DBF9901A282218
:1016A700C2AF121728121702901A00740E1216EE04
:1016B700A374061216EEA374151216EE901A037889
:1016C700807B0A1216EDA308DBF9901A0F788C7B42
:1016D700191216EDA308DBF912173B121719901A06
:1016E7002822E493F622E6438F01538FFD75EF021C
:1016F70075B7A575B7F1F0538FFE22438F02438F5D
:101707000175EF0275B7A575B7F1901A0DF0538FF4
:10171700FC22901A0D74A5D1EE901A0E745AD1EED0
:10172700227A3079D07820901A40D1E9E520F7095C
:10173700A3DAF7227A3079D0901A40E7D1EE09A3DD
:10174700DAF922AB74A875BB01027980BB02027972
:1017570081BB03027982BB04027994BB05027983BA
:10176700BB06027986BB07027992BB08027987BB61
:101777000902799CBB0A027988BB0B027989E8F7D1
:10178700227C05120562DCFB22C2AF12057212052C
:101797007912058012058712055312057212057911
:1017A7001205801205871205531205721205791268
:1017B7000580120587D2AF22C2AF120587120580B6
:1017C7001205791205721205531205871205801248
:1017D7000579120572120553120587120580120545
:1017E70079120572D2AF22AE74AF75C2AF1205720D
:1017F700120572120572120553DEF21205871205E1
:1018070053DFF8D2AF221217901217881217887574
:1018170074017575017576001217EE7C05AD5C12C3
:101827000562C3ED955C70F5C3E55C9401400AC39E
:10183700E55C94FF403702185112174A1216A71297
:101847001790C2AF75EF12121788DCD10576C3E582
:10185700769403500280C11217880575E5741490B9
:0D186700009F93F808C3E57598500280A813
:101874001217881217880574C3E574940C500280FB
:0F18840094120FE51216A7C2AF75EF1212178854
:0319FD000211567E
:101A00000E061507070104FFFF09020101A55A018F
:101A100000B4FFFFFF03FF01FF25D078C804FF01DA
:091A200000FF0A010100FF00FFB4
:101A400023484B696E673335412320202020202016
:101A500023424C48454C4923463333302320202031
:101A60002020202020202020202020202020202076
:101C0000C2AFC2D353D9BF7581C043B20343FF8073
:101C1000752438752503B1C975EF0275E24043F1AB
:101C20001053A4EF75D4FFD2847DFA780379E67C53
:101C300010752200752300901DD67B0675249875BB
:101C400025013084028142208408D8FBD9F9DCF7D1
:101C500081B4308408D8FBD9F9DCF781B4B189E4C8
:101C600093A3C39A6004DDC381B4DBDBB17B600264
:101C7000812B7B08E493FAA3B15CDBF87A30B15C8A
:101C8000752200752300B17BEAFCEBFDC3ED94FEE9
:101C9000400EB17B8A278B28ED30E0048A828B834B
:101CA000B17B7AC270D8C3ED94FE601350CEBD00F4
:101CB00025EC60097520007521FF0200008100A855
:101CC00027A9280809D804D90281D3B17FEA89AAB3
:101CD000F281C50D81A0C3ED94035049EDA2E092BD
:101CE000007AC5C3E5829400E583941C50902000DF
:101CF00010438F02438F0175B7A575B7F1F030001F
:101D00001FA827A9280809438F01538FFDD804D99C
:101D100002A12089AAE275B7A575B7F1F0A3A10DBC
:101D2000538FFC817C7AC1BD030CE493A3FAB140CC
:101D3000DCF8B138817C817EAA22AB23B15CEBFA5E
:101D4000EA6222752608C3E52313F523E52213F57D
:101D50002250066323A0632201D526EAB1C9B1C986
:101D600075260AEAF4200102D284300102C284B14D
:101D7000C9C3134002C201D526EB22B17FEAFB2082
:101D80008402A17F308402A184752608AE24AF2589
:101D9000C3EF13FFEE13FEB1CDB1C9C3EA13308414
:101DA000024480FA30E703632201C3E52313F523DD
:101DB000E52213F52250066323A0632201D526D91C
:101DC000E52265236523F52222AE24AF250E0FDE22
:101DD000FEDFFCD20122424C48656C693437316326
:041DE000F3300601D5
:00000001FF
